:1000000010C028C027C026C05DC024C023C022C0A5
:1000100021C020C01FC01EC01DC01CC01BC01AC0F4
:1000200019C011241FBECFEDCDBF10E0A0E6B0E097
:10003000ECE9F1E002C005900D92A236B107D9F7C4
:1000400020E0A2E6B0E001C01D92A436B207E1F7BD
:100050009AD0A2C0D5CF8FEF8ABB83E087BB81B592
:10006000866081BD81B5806481BD789485B7877EC7
:10007000806185BF379880B18F6080B908959C01F9
:1000800080958BBB98B322273170232F2095892F21
:100090008160822388BB0895C19A8FE097E201971F
:1000A000F1F700C00000C198089586B3847090E015
:1000B000089521B530E0287C87729927282B392BA9
:1000C00021BD08951F920F920FB60F9211242F9306
:1000D0003F934F935F936F937F938F939F93AF93D0
:1000E000BF93EF93FF93209162003091630081E012
:1000F00090E002C0880F991F2A95E2F7C0DFCCDF9D
:1001000080916200909163000196909363008093C8
:1001100062008091620090916300099724F0109230
:10012000630010926200B29B0CC0809160009091BD
:100130006100019731F086E090E0BBDF81E090E064
:100140000DC0B2990FC0809160009091610002973C
:1001500049F085E090E0ADDF82E090E090936100AF
:1001600080936000FF91EF91BF91AF919F918F912C
:100170007F916F915F914F913F912F910F900FBEA3
:100180000F901F90189567DF85B7806285BF8895AF
:0C01900085B78F7D85BFF8CFF894FFCFB6
:02019C00010060
:00000001FF
